:020000040800F2
:1000000000070020F10100088D26000845260008A1
:100010006D2600084526000865260008F301000843
:10002000F3010008F3010008F30100081537000888
:10003000F3010008F3010008F3010008F3010008D0
:10004000F3010008F3010008F3010008F3010008C0
:10005000F3010008F3010008093A0008313A0008EA
:10006000593A0008813A0008A93A0008F30100084B
:10007000F3010008F3010008F3010008F301000890
:10008000F3010008F3010008F3010008F301000880
:10009000F30100082526000835260008D13A00089B
:1000A000F3010008F3010008F3010008F301000860
:1000B000A53B0008F3010008F3010008F301000864
:1000C000F3010008F3010008F3010008F301000840
:1000D000F3010008F3010008F3010008F301000830
:1000E000353B0008F3010008F3010008F3010008A4
:1000F000F3010008F3010008F3010008F301000810
:10010000F3010008F3010008F3010008F3010008FF
:10011000F3010008F3010008F3010008F3010008EF
:10012000F3010008F3010008F3010008F3010008DF
:10013000F3010008F3010008F3010008F3010008CF
:10014000F3010008F3010008F3010008F3010008BF
:10015000F3010008F3010008F3010008F3010008AF
:10016000F3010008F3010008F3010008F30100089F
:10017000F3010008F3010008F3010008F30100088F
:10018000F3010008F3010008F3010008F30100087F
:10019000F3010008F3010008F3010008F30100086F
:1001A000F3010008F3010008F3010008F30100085F
:1001B000F3010008F3010008F3010008F30100084F
:1001C000F3010008F3010008F3010008F30100083F
:1001D000F3010008F3010008F3010008F30100082F
:1001E0005D0F00080000000000000000000000009B
:1001F00002E000F000F8FEE772B6374880F30888A6
:10020000364880F3098836483649086040F20000D5
:10021000CCF200004EF63471CEF200010860BFF35C
:100220004F8FBFF36F8F40F20000C0F2F0004EF628
:100230008851CEF200010860BFF34F8FBFF36F8F7C
:100240004FF00000E1EE100A4EF63C71CEF20001D4
:100250000860062080F31488BFF36F8F04F03CF928
:1002600004F01CFA4FF055301F491B4A91423CBF25
:1002700041F8040BFAE71D49184A91423CBF41F886
:10028000040BFAE71A491B4A1B4B9A423EBF51F82E
:10029000040B42F8040BF8E700201849184A914271
:1002A0003CBF41F8040BFAE704F01AF904F03CFAF9
:1002B000144C154DAC4203DA54F8041B8847F9E797
:1002C00000F042F8114C124DAC4203DA54F8041B12
:1002D0008847F9E704F002B9000700200023002056
:1002E0000000000808ED00E00001002000070020E9
:1002F000C849000800230020A4230020A8230020D0
:1003000054510020E0010008E4010008E401000865
:10031000E40100082DE9F04F2DED108AC1F80CD052
:10032000C3689D46BDEC108ABDE8F08F002383F3BF
:1003300011882846A047002003F072FDFEE703F075
:10034000FBFC00DFFEE70000F8B500F019FE04F04A
:1003500065F8074604F0B6F80546C0BB294B9F4236
:1003600035D001339F4235D0274B27F0FF029A4208
:1003700033D1F8B200F03AFC2E4642F2107400F08D
:100380003BFC08B10024264601F0EEF848B30320F8
:1003900000F03EF80024264635B11C4B9F4203D0A6
:1003A00004F088F800242646002004F041F80EB13D
:1003B00000F044F800F054FC02F070F90546C4B9AE
:1003C00000F096FC4FF47A7003F030FDF7E72E460C
:1003D0000024D4E704460126D1E7064640F6C414BB
:1003E000CDE740F6C4139C4204BF4FF47A74012653
:1003F000D2E702F053F9431BA342E1D900F01EF803
:10040000DAE700BF010007B0000008B0263A09B0E3
:10041000084B187003280CD8DFE800F00805020824
:10042000022000F009BE022000F0FEBD024B0022B7
:100430005A607047A8230020AC23002010B501F0BB
:1004400093F830B1234B03221A70234B00225A60D9
:1004500010BD224B224A1C4619680131F8D00433E2
:100460009342F9D16268A242F2D31E4B9B6803F11A
:10047000006303F510439A42EAD203F0EDFF03F064
:10048000FFFF002000F096FD0220FFF7C1FF164B92
:100490009A6D00229A65996F9A67996FD96DDA659E
:1004A000D96FDA67D96F196E1A66D3F88010C3F85E
:1004B0008020D3F8803072B64FF0E0233021C3F8AB
:1004C000084DD4E9003281F311889D4683F30888F2
:1004D0001047BDE7A8230020AC23002000900008AF
:1004E000209000080023002000100240094A1368F1
:1004F00049F2690099B21B0C00FB01331360064BF3
:10050000186844F2506182B2000C01FB02001860CE
:1005100080B27047142300201023002010B5002162
:100520001022044600F0A2FD034B03CB2060616063
:100530001868A06010BD00BF9075FF1FF0B5ADF545
:10054000517D6EAC4FF4C47207460D462046002123
:1005500000F08CFD02F0A2F8244B4FF47A72B0FB4D
:10056000F2F0186093E80700022384E807000DF515
:10057000ED702382FFF7D2FF4BF214531C49238402
:1005800006A804F037F9202384F832310DF2EB2667
:1005900006AB0DF1380C1A4603CA62453060716033
:1005A000134606F10806F6D10FAE31460122204669
:1005B00000F0A8FD00230393AB7E029305F119031D
:1005C000019380B20123CDE904600093E97E05A385
:1005D000D3E90023384602F06DFC0DF5517DF0BDE6
:1005E000AFF300809E6AC421818A46EEB4230020C6
:1005F000044800082DE9F0412C4C237ADAB08046FB
:100600000D465BBB27A9284600F0A2FE074600283E
:1006100042D19DF89D60C82E3ED801464FF4A66297
:10062000204600F023FD4FF48073C4F8F8314FF4F6
:100630000073C4F80C334FF44073C4F820343246CE
:100640000DF19E0104F1090000F0FEFC26449DF826
:100650009C30777223720BB9EB7E237281220021CA
:1006600006AC27A800F002FD0122214627A800F0D1
:10067000B5FE00230393AB7E029305F1190380B20C
:1006800001932823CDE904400093E97E05A3D3E933
:100690000023404602F00EFC5AB0BDE8F08100BFD6
:1006A000AFF3008026417272DF25D7B7FC330020FC
:1006B000F0B5254E4FF48A7505FB0065F1B096F84C
:1006C000D83085F8DC300024D822214685F8E8406F
:1006D0003AA800F0CBFC06F1090000F0BFFCD5F809
:1006E000E4308DF8F000C2B206AF06F109010DF159
:1006F000F100CDE93A3400F0A7FC394601223AA8CE
:1007000000F0A2FE80B2CDE9047008230127CDE9F4
:10071000023706F1D803019330230093317A0B4856
:1007200007A3D3E9002302F0C5FBA04206DD01F0D8
:10073000B5FFC5F8E000384671B0F0BD2046FBE7D4
:1007400078F6339F93CACD8DFC330020CC33002044
:100750002DE9F0411D4D1E4E1E4F86B0284602F079
:10076000D5FB034658B30024CDE90344ADF814404B
:10077000027B8DF8142099684068029403AA03C292
:100780001B68DFF8548043F00043029301F088FFB8
:10079000821941F10003009402A9384601F0E0F803
:1007A000A04205DD284602F0B5FB88F80040D5E7F9
:1007B00098F80030072B05D8013388F8003006B0D0
:1007C000BDE8F081014802F0A5FBF8E7CC3300203A
:1007D00040420F00383900203139002070B50D46F5
:1007E00014461E4602F0C2FA50B9022E10D1012C56
:1007F0000ED112A3D3E90023C5E90023012007E0AD
:10080000282C10D005D8012C09D0052C0FD00020A1
:1008100070BD302CFBD10BA3D3E90023ECE70BA375
:10082000D3E90023E8E70BA3D3E90023E4E70BA314
:10083000D3E90023E0E700BFAFF30080401DA12013
:1008400026812A0B78F6339F93CACD8D9E6AC421E8
:10085000818A46EE26417272DF25D7B7F017304AFB
:1008600039059E5638B505460E4C0021013500F07D
:10087000C3FBA4F82C55B4F82C0500F0A5FB78B107
:10088000B4F82C0500F0B0FB014648B9B4F82C05CB
:1008900000F0B2FBB4F82C350133A4F82C35EAE7AC
:1008A00038BD00BFFC33002010B50A4B0A4A1A605D
:1008B00003F5805393F858203AB95C6D2CB120466B
:1008C00000F0D0FE204601F007F8BDE810400348D4
:1008D00000F0C8BE38390020584800087849002088
:1008E0002DE9F04F8FB000AF05460C4602F03EFAFE
:1008F00000284BD1237E022B1BD1E38A012B18D178
:1009000001F0CCFE0646FFF7F1FD03464FF4C87038
:10091000DFF8D482B3FBF0F206F5167602FB103353
:1009200016FA83F3C8F80030E37E33B9A74B0022F0
:100930001A703C37BD46BDE8F08F07F12401204610
:1009400000F0BAFC0028F4D107F11400FFF7E6FD2F
:1009500097F8264007F11401224607F1270003F01B
:1009600017FF0028E2D10F2C08D8984B1C70D8F83C
:100970000030A3F51673C8F80030DAE797F82410B2
:100980000029D6D0284602F0E9F9D2E7E38A282BDD
:1009900033D010D8012B2BD0052BCAD1BFF34F8FEA
:1009A0008B498C4BCA6802F4E0621343CB60BFF3FF
:1009B0004F8F00BFFDE7302BBBD1874EE17E327AEF
:1009C0009142B6D1607E3146002291F8DC508542DA
:1009D00000F0AD800132042A01F58A71F5D1326848
:1009E00040F6B831FA328A4294BF32603160A0E7F3
:1009F00021462846FFF7A2FD9BE721462846FFF740
:100A0000F9FD96E7B2F8EC507B6005F103094FEA77
:100A100099094FEA8902D11DC908A8EBC1039D4677
:100A2000EB460021584600F021FB04F1EE012A4676
:100A30003144584600F008FB7B6813B9012000F0F0
:100A4000B9FA96F8D20000F0BFFA044630B9307215
:100A500000F0DAFA204600F0ADFAB0E0D6F8D42083
:100A60003AB996F8D200B6F82C25824201D8FFF7A1
:100A7000F9FED6F8D4202A44944208D296F8D2003F
:100A8000B6F82C250130824201D8FFF7EBFE7068E2
:100A90005FFA89F2594600F0F1FA08B9C54679E0E3
:100AA000726896F8D2002A447260D6F8D42005EB1A
:100AB0000209C6F8D49000F087FA814509D396F868
:100AC000D220D6F8D4000132001B86F8D220C6F816
:100AD000D400FF2D0FD80024347200F095FA204680
:100AE00000F068FA00F040FD3C4B188108B9FFF7B0
:100AF000A5FCC5461DE7BB6896F8D9000AFB036252
:100B0000FB68D2F8E41082F8E83001F58061C2F8A1
:100B1000E030C2F8E410FFF7CBFDFFF719FE96F8BE
:100B2000D920013202F0030286F8D920B6E74FF44B
:100B30008A7A0AFB02F505F1EA013144204600F009
:100B4000B7FCF86000287FF4F4AE3544012285F844
:100B5000E82001F0A3FDD5F8E020D6ED007ADFED26
:100B6000206A801A192838BF192040F6B8329042FE
:100B700028BF1046B8EE677A07EE900AF8EEE77ADB
:100B800067EEA67ADFED176AE7EE267AFCEEE77AE3
:100B9000C6ED007A96F8D9307168BB600AFB03F4A1
:100BA000321992F8E8505DB1D2F8E4308B42E84651
:100BB0003FF428AF002182F8E810C2F8E010C546E3
:100BC0007368064A9B0A01331381B2E6C5330020DD
:100BD00000ED00E00400FA05FC330020B4230020FF
:100BE000CDCCCC3D6666663FC8330020014B187003
:100BF000704700BFC023002038B54FF00054144B9D
:100C000022689A4221D1607DF0B1124B12491870CE
:100C10001248237D03724FF48073C0F8F8314FF40B
:100C20000073C0F80C3300254FF44073C0F8203433
:100C3000C0F8E450C922093000F006FAE022294643
:100C4000204600F013FA012038BD0020FCE700BF69
:100C50009AAD44C5C023002016000020FC330020BC
:100C600037B500F081FC194D1949288102236B71B9
:100C700000220123174801F0EDF800230193164BE1
:100C8000164900931648174B4FF4805202F03EF875
:100C9000154B197811B1124802F060F801F0FEFC12
:100CA0000446FFF723FC4FF4C873B0FBF3F202FBDA
:100CB000130304F5167010FA83F00C4B186003F060
:100CC00001FC08B10F232B8103B030BDB4230020F9
:100CD00040420F0038390020DD070008C4230020FF
:100CE000CC330020E1080008C0230020C8330020D6
:100CF0002DE9F04F2DED028B90A7D7E900670FF299
:100D00004429D9E90089884C95B00DAD9FED848BBD
:100D1000FFF71EFDDFF834B200230C93ADF83C3032
:100D20000D936B6000230DF125028DED008B4FF0CC
:100D3000010A09A958468DF825308DF824A001F044
:100D400015FC9DF824200023002A40F0AF802046A7
:100D500002F00CF80546002847D1DFF8F4B101F0A5
:100D60009DFCDBF8003098423FD301F097FC0790E0
:100D7000FFF7BCFB079A4FF4C873B0FBF3F101FB1C
:100D8000130302F5167010FA83F0CBF80000DFF8B9
:100D9000C4B19BF800100791002914BF2B4653469D
:100DA00010A88DF83030FFF7B9FB0799C1F1100298
:100DB000D2B2062A10AB28BF062219440DF1310029
:100DC000079200F041F9079A0CAB039318230293A2
:100DD0000132564BD2B2CDE900A304923B463246D3
:100DE000204602F009F88BF8005001F057FC504AF9
:100DF000504D1368C31AB3F57A7F32D3106001F0F7
:100E00004FFC02460B46204602F08EF8204601F0C9
:100E1000ADFF30B32B7ADFF840A1002B14BF0323C2
:100E200002238AF8053001F039FC0DF1400B4FF434
:100E30007A730122B0FBF3F05946CAF8000050461D
:100E400000F012FA182302933B4B019380B240F258
:100E50005513CDE903B0009342464B46204601F0BE
:100E6000CBFF2B7AB3B101F019FC4FF0000A834697
:100E70004FF48A7295F8D900504400F0030002FB49
:100E8000005393F8E810002934D00AF1010ABAF1AE
:100E9000040FEFD1C82002F0C9FF2B7A002B7FF49A
:100EA00034AF15B0BDEC028BBDE8F08F4FF0904130
:100EB00010A84A6982F010024A611946102200F017
:100EC000D5F80DF126030AAA0CA9584600F06EFECB
:100ED00095E8030011AB83E803009DF83C308DF8E2
:100EE0004C300C9B109310A9DDE90A23204602F038
:100EF000EFF917E7D3F8E01049B12B68FA2B38BFA8
:100F0000FA23ABEB01010533B1EB430FBDD3FFF780
:100F1000CFFB4FF48A720028B7D1BBE7AFF3008054
:100F20000000000000000000CC330020C43300208B
:100F30002C390020FC33002030390020401DA12036
:100F400026812A0BF1C6A7C1D068080F38390020C6
:100F5000C8330020C5330020B423002008B505485D
:100F600000F0C8FEBDE80840034A0449002003F031
:100F7000F3BB00BF38390020404E0020A90800080C
:100F800070B503F0EFF8094E094D30800024286851
:100F90003388834208D903F0E1F82B680444013315
:100FA000B4F5104F2B60F2D370BD00BF344E00205B
:100FB000084E002003F088B900F10060920000F5AF
:100FC000104003F00BB90000054B1A68054B1B8855
:100FD0009B1A834202D9104403F0C0B80020704726
:100FE000084E0020344E0020024B1B68184403F0CA
:100FF000BBB800BF084E0020024B1B68184403F02A
:10100000C5B800BF084E0020064991F8243033B11E
:101010000023086A81F824300822FFF7CDBF0120A1
:10102000704700BF0C4E0020022802BF4FF09043D3
:1010300010229A6170470000022802BF4FF09043CF
:101040004FF480129A61704710B50023934203D089
:10105000CC5CC4540133F9E710BD000003460246DE
:10106000D01A12F9011B0029FAD170470244034635
:10107000934202D003F8011BFAE770472DE9F843C9
:101080001F4D144695F824200746884652BBDFF8CA
:1010900070909CB395F824302BB92022FF2148464C
:1010A0002F62FFF7E3FF95F82400C0F10802A24287
:1010B00028BF2246D6B24146920005EB8000FFF7DA
:1010C000C3FF95F82430A41B1E44F6B2082E174423
:1010D0009044E4B285F82460DBD1FFF795FF002847
:1010E000D7D108E02B6A03EB82038342CFD0FFF70E
:1010F0008BFF0028CBD10020BDE8F8830120FBE75F
:101100000C4E00202DE9F3470D4604460021904681
:10111000284640F27912FFF7A9FF2346202200213A
:10112000284602F077F8231D02222021284602F0EB
:1011300071F8631D03222221284602F06BF8A31DDB
:1011400003222521284602F065F804F10803102245
:101150002821284602F05EF804F110030822382105
:10116000284602F057F804F11103082240212846CE
:1011700002F050F804F1120308224821284602F038
:1011800049F804F1140320225021284602F042F8C5
:1011900004F1180340227021284602F03BF804F1C4
:1011A00020030822B021284602F034F804F121037C
:1011B0000822B821284602F02DF804F12207C026A3
:1011C0003B46314608222846083602F023F8B6F599
:1011D000A07F07F10107F3D194F832308DF8073082
:1011E00031460DF107030822284602F013F80026C5
:1011F00004F1330A9DF807304FEAC6099E4209F50B
:10120000A47720D394F83231502B28BF50238DF887
:101210000730B8F1000F08D139460DF10703072256
:10122000284601F0F7FF09F24F17002604F23314A5
:101230009DF807309E4207EBC6010DD30731C80861
:1012400002B0BDE8F0870AEB0603082239462846BB
:1012500001F0E0FF0136CDE7A3190822284601F08E
:10126000D9FF0136E4E7000013B504460846002123
:1012700001602346C0F803102022019001F0CAFF4C
:101280000198231D0222202101F0C4FF0198631D53
:101290000322222101F0BEFF0198A31D0322252174
:1012A00001F0B8FF019804F108031022282101F091
:1012B000B1FF072002B010BDF7B5047F05460E460A
:1012C0002CB1838A122B02D9012003B0F0BD002378
:1012D000194607220096284601F060FE731C009311
:1012E000012200230721284601F058FED4B9B31C7F
:1012F0000093052223460821284601F04FFE0D24C5
:10130000B378102BE0D83746B278BB1B934210D38A
:101310002B7FA88A0734E408B3B9844294BF002025
:101320000120D2E7AB8ADB00083BDB08B37008245E
:10133000E6E7FB1C0093214600230822284601F023
:101340002DFE08340137DFE7201A18BF0120BCE763
:10135000F7B5047F05460E462CB1838ACA2B02D905
:10136000012003B0F0BD002319460096082228464C
:1013700001F014FE731CD4B90822009311462346D1
:10138000284601F00BFE10247378C82BE8D80123FF
:1013900072785F1C013B934210D32B7FA88A0734DD
:1013A000E408B3B9844294BF00200120D9E7AB8A96
:1013B000DB00083BDB0873700824E5E7F3190093B2
:1013C000214600230822284601F0E8FD08343B4668
:1013D000DEE7201A18BF0120C3E70000F7B50D466D
:1013E00004460021164628468122FFF73FFE234689
:1013F00008220021284601F00DFF94F901206378AE
:10140000002AB8BF7F238DF807309EB90DF107037E
:1014100007220821284601F0FDFE0F27002602348E
:101420009DF807309E4207EBC60105D30731C80877
:1014300003B0F0BD0827F1E7A3190822284601F000
:10144000E9FE0136ECE70000F7B50E46054600213F
:1014500014463046CE22FFF709FE2B4628220021F3
:10146000304601F0D7FE2B7AC82B28BFC8238DF851
:1014700007308CB90DF1070308222821304601F00E
:10148000C9FE30242F469DF807207B1B934205D3CD
:10149000E01DC00803B0F0BD2824F3E707F10903FD
:1014A00021460822304601F0B5FE08340137EAE74C
:1014B000F7B5047F05460E4634B1838AB3F5827FC3
:1014C00002D9012003B0F0BD0096012310220021B3
:1014D000284601F063FDDCB9B31C009309222346C2
:1014E0001021284601F05AFD19247388B3F5807F36
:1014F000E7D837467288BB1B934210D32B7FA88A4C
:101500000734E408B3B9844294BF00200120D9E72E
:10151000AB8ADB00103BDB0873801024E5E73B1D42
:101520000093214600230822284601F037FD0834A5
:101530000137DFE7201A18BF0120C3E730B5094D96
:101540000A4491420DD011F8013B5840082340F362
:101550000004013B2C4013F0FF0384EA5000F6D155
:10156000EFE730BD2083B8EDF7B5384A1068516811
:101570006B4603C36A4636493648082303F018F918
:101580000446002833D10A25334A106851686B4657
:1015900003C36A4631492F48082303F009F904467A
:1015A000002849D00369B3F55C3F45D8B0F8661010
:1015B00041F2B54291423FD1294A024402F15C0115
:1015C0008B4239D35C3B234900209E1AFFF7B6FFBC
:1015D0003246074604F164010020FFF7AFFFA3681D
:1015E0009F4229D1E368984208BF002524E003699F
:1015F000B3F55C3F27D8418B41F2B542914220D1EF
:10160000174A024402F110018B4218D3103B1149D2
:1016100000209D1AFFF792FF2A46064604F11801A2
:101620000020FFF78BFFA3689E4202D1E368984237
:1016300001D00D25A8E70025284603B0F0BD1025F0
:10164000A2E70C25A0E70B259EE700BF284800086D
:10165000DC6F03000090000831480008906F030021
:101660000870FFF710B5037C044613B9006803F057
:1016700087F8204610BD00000023BFF35B8FC360D6
:10168000BFF35B8FBFF35B8F8360BFF35B8F7047EC
:10169000BFF35B8F0068BFF35B8F704770B5054683
:1016A0000C30FFF7F5FF05F1080604463046FFF75A
:1016B000EFFFA04206D930466D68FFF7E9FF2544E9
:1016C000281A70BD3046FFF7E3FF201AF9E7000043
:1016D00070B50546406898B105F10800FFF7D8FFDE
:1016E00005F10C0604463046FFF7D2FF844230462F
:1016F00094BF6D680025FFF7CBFF013C2C44201AF6
:1017000070BD000038B50C460546FFF7C7FFA04284
:1017100010D305F10800FFF7BBFF04446868B4FB71
:10172000F0F100FB1144BFF35B8F0120AC60BFF30D
:101730005B8F38BD0020FCE72DE9F04114460746D9
:101740000D46FFF7C5FF844228BF0446D4B1B84612
:1017500058F80C6B4046FFF79BFF3044286040462A
:101760007E68FFF795FF331A9C4203D86C60012016
:10177000BDE8F0816B60A41B3B68AB602044E8606F
:101780000220F5E72046F3E738B50C460546FFF79B
:101790009FFFA04210D305F10C00FFF779FF04442E
:1017A0006868B4FBF0F100FB1144BFF35B8F0120CC
:1017B000EC60BFF35B8F38BD0020FCE72DE9FF41F3
:1017C000884669460746FFF7B7FF6C4606B204EB4A
:1017D000C6060025B44209D06268206808EB0501FE
:1017E000FFF732FC636808341D44F3E729463846A6
:1017F000FFF7CAFF284604B0BDE8F081F8B50546FA
:101800000C300F46FFF744FF05F10806044630464A
:10181000FFF73EFFA042304688BF6C68FFF738FFF5
:10182000201A386020B130462C68FFF731FF204481
:10183000F8BD000073B5144606460D46FFF72EFFAF
:10184000844228BF04460190DCB101A93046FFF76D
:10185000D5FF019B33B93268C5E90233C5E90024DD
:1018600001200CE09C4238BF019428600198686018
:101870008442F5D93368AB60241AEC60022002B0D0
:1018800070BD2046FBE700002DE9FF410F46694689
:10189000FFF7D0FF6C4600B204EBC0050026AC4257
:1018A00009D0D4F8048054F8081BB8194246FFF751
:1018B000CBFB4644F3E7304604B0BDE8F0810000BE
:1018C00038B50546FFF7E0FF044601462846FFF716
:1018D00019FF204638BD000008B102F051BF704723
:1018E0007047000010B41346026814680022A44632
:1018F0005DF8044B6047000000F5805090F86904E3
:101900007047000000F5805090F8620470470000B6
:1019100000F5805090F9680470470000502070472F
:10192000302383F3118800F58052D2F8AC34D2F81A
:10193000A8041844D2F8A4341844D2F88C341844BB
:10194000D2F89C341844D2F898341844002383F316
:101950001188704700F58050C0F86414012070476A
:101960002DE9FF470C4600F58051054691F86204C9
:10197000BDF8308098B1D1F888040130C1F88804EE
:101980002068860006D4207B08280BD9667B0EB120
:101990000F2807D9D1F88C340133C1F88C344FF0BB
:1019A000FF30AAE0302080F31188E86BD0F8C470D3
:1019B00017F4001713D0D1F890040130C1F8900447
:1019C000D1F89414002940F09B80CDF80080214686
:1019D000284600F0ADFE002383F311888DE0D0F897
:1019E000C460686BC6F301464FF0480919FB06094D
:1019F00020680028B4BF40F0804C4FEA804CC9F802
:101A000000C02068400044BF4CF00050C9F80000FE
:101A100094F80CC0300640EA0C40C9F8040094F871
:101A20000DC04FEA461ABCF1000F27D040F4401019
:101A3000C9F80400D1F8C0040130C1F8C00405EBB6
:101A40000A0101F58351087F40F020000877207BD0
:101A5000CDE9022300F0BEFEDDE902230330801051
:101A6000F9B2814207F1010710DA04EB810C09EBAE
:101A70008101DCF804C0C1F808C0F1E705EB0A01F8
:101A800001F58351087F6CF34510DFE7E96B012016
:101A9000B040C1F8CC0006F1830105EB4111C1E96A
:101AA000002305EB461101F583512046083104F16E
:101AB0000C0750F804CB41F804CBB842F9D10088A8
:101AC0000880AA4441F278014AF801600AF5805A78
:101AD00008F003019AF87C0041F0100120F01F008B
:101AE00001438AF87C10002181F31188CDF8008031
:101AF0002146284600F01CFE012004B0BDE8F08716
:101B0000002068E738B5C26B936923F00103936145
:101B1000044600F0C3FD0546E36B9B69DB0706D571
:101B200000F0BCFD431BFA2BF6D9002004E004F5BD
:101B30008054012084F8620438BD000013B500F51C
:101B400080540191606DFFF7C3FD1F280AD90199E8
:101B5000606D2022FFF732FEA0F120035842584169
:101B600002B010BD0020FBE708B5302383F31188D5
:101B700000F58050406DFFF77FFD002383F311884F
:101B800008BD0000002202608281426082607047CE
:101B900010B500220023C0E900230023044603817E
:101BA0000C30FFF7EFFF204610BD00002DE9F04795
:101BB0009A4688B0074688469146302383F31188B9
:101BC00007F580546846FFF7E3FF606DFFF766FD99
:101BD0001F282DD9606D20226946FFF771FE20284D
:101BE00026D194F862341BB303AD444605AB2E46B0
:101BF00003CE9E4220606160354604F10804F6D1B0
:101C000030682060B388A380DDE90023C9E90023A0
:101C1000BDF80830AAF80030002383F3118853463A
:101C20004A464146384608B0BDE8F04700F044BD9A
:101C3000002080F3118808B0BDE8F0872DE9F84F47
:101C4000064635468846182200210430FFF70EFA72
:101C5000254B45F8403B06F582572C46204620345C
:101C6000FFF796FFA742F9D106F580544FF4805351
:101C700025640025C4E9113501236765E56484F80E
:101C8000503084F8583006F5845706F5A4594FF0C3
:101C9000000A4FF0000B47E908ABA7F11800FFF767
:101CA00071FF203747F8285C4F45F4D184F86884E9
:101CB000A4F86A54A4F86C54A4F86E5484F87054D0
:101CC000A4F87254A4F87454A4F8765484F87854A0
:101CD000B8F1000F02D0054800F0DAFC044BF363C2
:101CE0003046BDE8F88F00BF584800083C4800085F
:101CF0000064004010B5044B197804464A1C1A7061
:101D0000FFF79CFF204610BD3D4E00202DE9F84313
:101D100015460C4600295CD0022001F06FFE2E49CA
:101D2000B0FBF4F78C428CBF0A2111214B1EB7FB8C
:101D3000F1F601FB1671DAB221B1022B1946F5D882
:101D4000002032E0731EB3F5806FF9D2C2EBC208F7
:101D500008F103014FEAE10EC1F3C701A2EB010C48
:101D60000EF101094FF47A735FFA8CF70EFB033E14
:101D700059FA8CFCBEFBFCFCBCF5617F17DC1FFA3A
:101D80008CF34A1C57FA82F27243B0FBF2F08442A1
:101D9000D6D14A1E0F2AD3D87A1E072AD0D80120BE
:101DA0002B806E8028716971AF71BDE8F88308F1EE
:101DB000FF314FEAE10CC1F3C701521A0CF1010ED9
:101DC000D7B20CFB03335EFA82F2B3FBF2F39BB2A1
:101DD000D7E70846E9E700BF3F420F0030B50D4B9B
:101DE0000D4D05201C786C438C420ED159785180E2
:101DF00099785171D9789171197911715B7903EBE7
:101E000083035B001380012030BD013803F106031A
:101E1000E8D1F9E79C48000840420F000B4B10B591
:101E20004FF45472044600211846FFF71FF9084B7F
:101E3000A3624033E362D8332363F0336363E36B1D
:101E400060620022C3F8C02010BD00BF00A40040A3
:101E500070A400402DE9F04700F580551F4695F825
:101E60006834012B88B004468946904604D9002680
:101E7000304608B0BDE8F087994A52F8231009B9F6
:101E800042F823009748C4F81C90017884F8207029
:101E900099B9302383F31188934B9A6D42F0007205
:101EA0009A659A6B42F000729A639A6B22F0007204
:101EB0009A630123037081F3118895F861647EB9F8
:101EC000302383F311880321152001F0ABFE032199
:101ED000162001F0A7FE012385F8613486F31188EE
:101EE000302383F31188E26B936923F0100393612D
:101EF00000F0D4FB8246E36B9E6916F0080609D019
:101F000000F0CCFBA0EB0A03FA2BF4D9002686F3F1
:101F10001188ADE79A6942F001029A6100F0BEFBB8
:101F20008246E36B9A69D00706D400F0B7FBA0EBBA
:101F30000A03FA2BF5D9E9E79A6942F002029A619D
:101F4000E36B4FF0000AC3F854A08AF31188686D60
:101F5000FFF792FB202200216846FFF787F802A8CE
:101F6000FFF710FE04F58353CDF818A06A463344FA
:101F70000DF1180E9446BCE80300F4451860596052
:101F8000624603F10803F5D1DCF800001860203642
:101F90009CF804201A71B6F5806FDBD1002304F59C
:101FA000A35285F8603485F863340A3249462046E6
:101FB000FFF7ACFE064690B9E26B936923F001038C
:101FC000936100F06BFB0546E36B9B69D9077FF5D6
:101FD0004EAF00F063FB431BFA2BF5D947E795F8AA
:101FE0006E34C5F87C94591E95F86F34E26B013B52
:101FF0001B0243EA416395F8701401390B43B5F8AD
:102000006C14013943EA0143D361B8F1000F36D0B3
:1020100004F5A352123241462046FFF7DFFE90B985
:10202000E26B936923F00103936100F037FB0546EF
:10203000E36B9B69DA077FF51AAF00F02FFB431BB8
:10204000FA2BF5D913E795F87724C5F88084511E4B
:1020500095F87824E36B013A120142EA012295F8DF
:10206000761401390A43B5F87414013942EA014281
:1020700042F40002DA60E36B4FF420629A64204677
:10208000FFF7CCFE002385F86934E36B6FF0404224
:102090001A65E36B154A5A65E36B44229A65E36B54
:1020A0000722C3F8DC20E36B03229742DA653FF492
:1020B000DFAEE26B936923F00103936100F0EEFA67
:1020C0000746E36B9B69DB0705D500F0E7FAC31B06
:1020D000FA2BF6D9CBE6012385F86234C8E600BFB7
:1020E000384E00203C4E0020001002409B000800AB
:1020F0002DE9F04F00F5A5578BB00546904699465F
:102100004FF0000B41F2780A1037EB6BD3F8D43064
:1021100023FA0BF3DC0753D505EB4B1151444FEA7F
:102120004B120B7918074BD405F58056D6F894342A
:102130000133C6F89434C7E900890B79990648BF82
:10214000D6F8C43405EB020148BF0133514448BFFF
:10215000C6F8C4340B7943F008030B71DB0724D5B0
:1021600096F863340BB302A8019205F58354FFF788
:102170000FFD019A0834144405AB04F1080C2068E3
:1021800061681A4603C2083464451346F7D12068D3
:102190001060A2889A800123ADF810302B68CDE939
:1021A00002891B6C02A928469847D6F8B834D6F89D
:1021B00064040133C6F8B83410B103681B6998474A
:1021C0000BF1010BBBF1200F9FD10BB0BDE8F08FDD
:1021D0002DE9F04F8DB004460F4600F061FA8246BB
:1021E0008946002F56D1E36BD3F89020920141BF6E
:1021F00004F58051D1F8A8240132C1F8A824D3F8FD
:102200009020160703D100200DB0BDE8F08FD3F861
:102210009050E66AC5F30125482303FB0566E846AE
:102220004046FFF7AFFC326851004ABF22F06043DE
:10223000C2F38A4343F00043920048BF43F0804317
:102240000093736813F400131FBF04F58052012339
:102250008DF80D30D2F8C8340EBF8DF80D30013333
:10226000C2F8C834F38803F00F038DF80C304FF038
:10227000000B9DF80C0000F0ADFA5FFA8BF398426A
:1022800020D9F2180CA90B44127A03F82C2C0BF16C
:10229000010BEEE7012FB6D1E36BD3F8982095013F
:1022A00041BF04F58051D1F8A8240132C1F8A82417
:1022B000D3F898201007A6D0D3F89850266BC5F312
:1022C0000125A9E7EFB9E36BC3F8945004A8FFF721
:1022D0005FFC98E80F0007AD07C52B800023ADF821
:1022E000183023682046CDE904A91B6C04A998473F
:1022F00004F5805458B1D4F8A0340133C4F8A034A4
:1023000082E7012F04BFE36BC3F89C50DEE7D4F8EB
:10231000A4340133C4F8A434012075E72DE9F04159
:1023200005460F4600F58054012639462846FFF73A
:102330004FFF10B184F86364F7E7D4F8B834D4F8E9
:1023400064040133C4F8B83420B10368BDE8F04137
:102350001B691847BDE8F081F0B5C36B1A6C12F425
:102360007F0F2BD000F580541B6CC4F8BC3441F2B5
:102370007805002347194FF0010C00EB43122A4463
:102380005E01117911F0020F15D0490713D4B95924
:10239000C66BD6F8C8E00CFA01F111EA0E0F0AD0AC
:1023A000C6F8D010117941F004011171D4F89C24C1
:1023B0000132C4F89C240133202BDED1F0BD000093
:1023C00010B5254C254B226802B338B31A6D12069E
:1023D0000ED580221A6500F063F950EA01020B461F
:1023E00002D0013861F1000302462068FFF780FE49
:1023F0001A4A136D1B032AD523684FF4002103F5F5
:1024000080531165012283F8692420E001221A65B6
:1024100008221A654FF480621A6510BD196DC8074D
:1024200002D4196D890705D50321196510460021CD
:10243000FFF774FF094B1A6D100702D41A6DD1060D
:1024400005D518221A6520680121FFF767FF20686B
:10245000BDE81040FFF780BF384E00200064004008
:1024600008B5302383F31188FFF776FF002383F349
:10247000118808BDC36BD3F8C40080F40010C0F30A
:102480004050704708B5302383F3118800F5805021
:10249000406DFFF703F9002383F3118843090CBF54
:1024A0000120002008BD000000F5805393F8692446
:1024B00062B1C16B8A6922F001028A61D3F8AC244F
:1024C0000132C3F8AC24002283F86924704700006D
:1024D0002DE9F743302181F31188002500F5835160
:1024E00041F2780E4FF0010800F5805C00EB4514D6
:1024F0007444267977071CD4F6061AD5D0F83C9098
:102500008E69D9F8C87008FA06F63E4211D04F68B5
:1025100001970F689742019F9F410AD2C9F8D06086
:10252000267946F004062671DCF898440134CCF88C
:1025300098440135202D01F12001D7D1002383F3E8
:10254000118803B0BDE8F083F8B51E460023137070
:102550000F4605461446FFF795FF80F001003870DE
:102560001EB12846FFF786FF2070F8BD2DE9F04F19
:1025700085B09946DDE90EA30D46029313780193C9
:1025800091F800B08046164600F08AF82B78044691
:102590000F4613B93378002B41D022463B464046C4
:1025A000FFF796FFFFF75CFFFFF77EFF4B463246D3
:1025B0002946FFF7C9FF2B7833B1BBF1000F03D0D9
:1025C000012005B0BDE8F08F337813B1019B002BDB
:1025D000F6D108F580530393029B544577EB030330
:1025E0001DD2039BD3F86404C8B10368AAEB0401AD
:1025F0001B6898474B46324629464046FFF7A4FFE2
:102600002B7813B1BBF1000FDAD1337813B1019BF2
:10261000002BD5D100F044F804460F46DCE700203B
:10262000CFE7000008B50020FFF7CAFEBDE808406C
:1026300001F0A4B808B50120FFF7C2FEBDE80840CC
:1026400001F09CB800B59BB0EFF3098168226846A1
:10265000FEF7FAFCEFF30583014B9B6BFEE700BF2F
:1026600000ED00E008B5FFF7EDFF000000B59BB0FE
:10267000EFF3098168226846FEF7E6FCEFF3058375
:10268000014B5B6BFEE700BF00ED00E0FEE70000E2
:102690000FB408B5029801F079FBFEE701F05ABECD
:1026A00001F03CBE0139C9B202299EBF00EBC10056
:1026B0000023C0E901337047F8B51B885B07054666
:1026C0000E4615D4044600F11807BC4210D06368CA
:1026D00053B12B682846DB6B9847A368C1B23246DA
:1026E000606898470834F0E7A368002BF1D1F9E758
:1026F0000120F8BD73B56C4684E80600014600224F
:102700004E68D5B26EB98E685EB900EBC200021D8C
:1027100094E80300013582E803001D70012002B037
:1027200070BD0132032A01F10801E9D10020F6E76A
:102730002DE9F04F89B00446BDF848700E460546B5
:1027400000F118084FF0000907F004074FF0000AE5
:102750004FF0000BA84538D06B680BB9AB684BB194
:1027600057B923682046DB6B9847AB68C1B2324645
:10277000686898470835EDE7B9F1000FFAD1CDE95F
:1027800000ABADF80890334603AA06F1080E1868AE
:1027900059689446ACE80300083373456246F6D1A5
:1027A0001868CCF800009B88ACF80430FFF778FF7D
:1027B0000423ADF808302368CDE900011B6C69469D
:1027C000204698474FF00109D4E7012009B0BDE841
:1027D000F08F0000082817D909280CD00A280CD03F
:1027E0000B280CD00C280CD00D280CD00E2814BFB0
:1027F0004020302070470C20704710207047142074
:102800007047182070472020704700002DE9F041E4
:10281000456A15B94162BDE8F0814B6823F0604715
:10282000C3F38A464FEAD37EC3F3807816EA2306C1
:1028300038BF3E46AC462B465A68BEEBD27F22F0EC
:1028400060440AD0002A18DAA40CB44217D19D4281
:102850000FD10D60DEE71346EEE7A74207D102F085
:102860008044C2F3807242450BD054B1EFE708D2E6
:10287000EDE7CCF800100B60CDE7B44201D0B442D4
:10288000E5D81A689C46002AE5D11960C3E7000024
:102890002DE9F047089D01F007044FEAD5082244CE
:1028A00005F0070500EBD1004FF47F49944201D1B8
:1028B000BDE8F08704F0070705F0070A57453E46D4
:1028C00038BF5646C6F10806111B8E4228BF0E4679
:1028D000E10808EBD50E415C13F80EC0B94029FAA7
:1028E00006F721FA0AF1FFB28CEA010147FA0AF76A
:1028F00039408CEA010C03F80EC034443544D5E766
:1029000080EA0120082341F2210201B2400000299F
:1029100080B203F1FF33B8BF504013F0FF03F4D18E
:102920007047000038B50C468D18A54200D138BD5F
:1029300014F8011BFFF7E4FFF7E7000042684AB113
:10294000136843604389818901339BB29942438173
:1029500038BF83811046704770B588B02022044686
:102960000D4668460021FEF781FB20460495FFF7DF
:10297000E5FF024658B16B46054608AE1C4603CC3F
:10298000B44228606960234605F10805F6D1104677
:1029900008B070BD082817D909280CD00A280CD017
:1029A0000B280CD00C280CD00D280CD00E2814BFEE
:1029B0004020302070470C207047102070471420B2
:1029C000704718207047202070470000082817D94A
:1029D0000C280CD910280CD914280CD918280CD97B
:1029E00020280CD930288CBF0F200E2070470920DA
:1029F00070470A2070470B2070470C2070470D204D
:102A0000704700002DE9F843078C072F04461ED9B4
:102A1000D0E9029800254FF6FF73C5F12006A5F115
:102A2000200029FA05F108FA06F628FA00F03143E9
:102A30000143C9B21846FFF763FF0835402D03462E
:102A4000EBD1E1693A46BDE8F843FFF76BBF4FF6BB
:102A5000FF70BDE8F883000010B54B6823B9CA8A3F
:102A600063F30902CA8210BD04691A681C6003611D
:102A7000C38A013BC3824A60EFE700002DE9F84FAB
:102A80001D46CB8A0F46C3F30901052981469246AC
:102A90000B4630D00020AAB207F11A049EB2042ED1
:102AA0001FFA80F80FD8904503F1010306D3FB8A83
:102AB0000A4462F30903FB8201201AE01AF800605D
:102AC000E6540130EAE79045F1D2A1F1050B1C2351
:102AD0007C68BBFBF3F203FB12BB1FFA8BF6002CE6
:102AE00045D14846FFF72AFF044638B978606FF0B1
:102AF0000200BDE8F88F4FF00008E6E70026066008
:102B00007860ADB24FF0000B454510D90AEB0803D1
:102B1000221D13F8011B9155B1B208F101081B29C0
:102B20001FFA88F82BD0454506F10106F1D8FB8A3B
:102B3000C3F30902154465F30903BCE7013292B2FD
:102B40001C462368002BF9D16B1F0B441C21B3FBDF
:102B5000F1F301339BB29A42D3D2BBF1000FD0D133
:102B60004846FFF7EBFE20B9C4F800B0BFE70122EA
:102B7000E7E7C0F800B05E4620600446C1E745457F
:102B8000D5D94846FFF7DAFE08B92060AFE7C0F8AC
:102B900000B0002620600446B6E700002DE9F04FA3
:102BA0002DED028B1C4683B05B6901920746884677
:102BB000002B00F0A780238C2BB1E269002A00F0E3
:102BC000A180072B35D807F10C00FFF7B7FE0546AB
:102BD00038B96FF00205284603B0BDEC028BBDE8A2
:102BE000F08F14220021FEF741FA228CE16905F1F1
:102BF0000800FEF729FA208C013080B2FFF7E6FECC
:102C0000FFF7C8FE013880B2208401302874636960
:102C1000228C1B782A4403F01F0363F03F0348F023
:102C200000411372384669602946FFF7EFFD012520
:102C3000D1E702339BB20722C18A0633B3FBF2F31A
:102C4000828A521A9BB292B29342C2D800F10C030C
:102C50004FF0000908EE103A4FF0800A4E464D46FC
:102C600018EE100AFFF76AFE83460028B1D014223E
:102C70000021FEF7FBF9002E3AD1019BABF808309A
:102C800002220BF1080E1FFA82FC0CF10100BCF1CC
:102C9000060F218C80B201D88E422BD3FFF796FE0F
:102CA000FFF778FE62691278013802F01F028E4247
:102CB00008BF4FF0400A42EA49121BFA80F14AEA83
:102CC000020A013048F0004281F808A08BF8100099
:102CD000CBF8042059463846FFF798FD238C013580
:102CE000B3422DB289F001094FF0000AB8D172E762
:102CF0000022C6E7E169895D0EF802100136B6B21E
:102D00000132C0E76FF0010565E70000F8B5154630
:102D10000E463022002104461F46FEF7A7F9069B07
:102D20006360B5F5001F079BA76034BF6A094FF6C3
:102D3000FF72A36297B2E66104F1100000239A4289
:102D400006D800230360A782E3822383E360F8BDF3
:102D50000660013330462036F1E7000003781BB9E6
:102D60004BB2002BC8BF017070470000007870475D
:102D7000F8B50C46C969074611B9238C002B37D129
:102D8000257E1F2D34D8387828BB228C072A2CD8D2
:102D9000268A36F003032BD14FF6FF70FFF7C2FDF2
:102DA00020F001003102400441EA0561400C41EA93
:102DB00040254FF6FF72234629463846FFF7EEFEC0
:102DC000002807DD626913780133DBB21F2B88BF4F
:102DD00000231370F8BD218A2D0645EA012505431D
:102DE0002046FFF70FFE0246E5E76FF00300F1E72C
:102DF0006FF00100EEE7000070B58AB00446164699
:102E00000021282268461D46FEF730F9BDF838300B
:102E1000ADF810300F9B05939DF840308DF81830B9
:102E2000119B07936946BDF84830ADF82030204625
:102E3000CDE90265FFF79CFF0AB070BD2DE9F041B6
:102E4000D36905460C4616460BB9138C5BBB377E1F
:102E50001F2F28D895F80080B8F1000F26D03046F3
:102E6000FFF7D0FD3378210241EAC33141EA08017E
:102E7000338A41EA076141EA03410246334641F0A1
:102E800080012846FFF78AFE00280ADD3378012BEF
:102E900007D1726913780133DBB21F2B88BF00237F
:102EA0001370BDE8F0816FF00100FAE76FF00300E6
:102EB000F7E70000F0B58BB004460D461746002139
:102EC000282268461E46FEF7D1F89DF84C305A1E5F
:102ED000534253418DF800309DF84030ADF810302A
:102EE000119B05939DF848308DF81830149B07937B
:102EF0006A46BDF85430ADF8203029462046CDE969
:102F00000276FFF79BFF0BB0F0BD0000406A00B1F6
:102F100004307047436A1A68426202691A600361AA
:102F2000C38A013BC38270472DE9F041D0F820806D
:102F3000194E14461D464146002709B9BDE8F081E7
:102F4000D1E90223A21A65EB0303964277EB030350
:102F50001ED2036A8B420DD1FFF77EFD036A1B6808
:102F6000036203690B60C38A0161016A013BC3828A
:102F70008846E2E7FFF770FD0B68C8F80030036988
:102F80000B60C38A0161013BC382D8F80010D4E70B
:102F900088460968D1E700BF80841E002DE9F04F04
:102FA0008BB00D46DDF8509014469B4680460028B5
:102FB00000F01981B9F1000F00F01581531E3F2B6D
:102FC00000F21181012A03D1BBF1000F40F00B8107
:102FD0000023CDE90833B8F81430B5EBC30F4FEA3E
:102FE000C30703D300200BB0BDE8F08F2B199F421D
:102FF000D8F80C303ABF7F1BFFB227461BB9D8F870
:103000001030002B7AD0272D4ED8C5F12806B742B4
:103010004FF000032CBFF6B23E4600932946D8F885
:10302000080008AB3246FFF733FCA7EB060A35442D
:103030005FFA8AFAB8F8143003F10053053BDB005D
:103040000493D8F80C3003932821039B13B1BAF1F1
:10305000000F2CD1D8F8100040B1BAF1000F05D004
:10306000009608AB5246691AFFF712FC38B2002FDF
:10307000B8D066070AD00AAB03EBD401624211F85C
:10308000083C02F00702134101F8083C082C3CD927
:10309000102C40F2B580202C40F2B780BBF1000F1D
:1030A00000F09C80082334E0BA460026C2E7049B67
:1030B000E02B28BFE02306930B44AB42059314D9C1
:1030C0005A1B03980096924534BF5246D2B2691AF1
:1030D00008AB04300792FFF7DBFB079A1644AAEB14
:1030E000020A1544F6B25FFA8AFA049B069A059919
:1030F0009B1A0493039B1B680393A6E70093D8F8DD
:10310000080008AB3A462946AEE7BBF1000F13D0E2
:103110000123B4EBC30F6CD0082C12D89DF82030DB
:10312000621E23FA02F2D50706D54FF0FF3202FAEB
:1031300004F423438DF820309DF8203089F80030C6
:1031400051E7102C12D8BDF82030621E23FA02F28B
:10315000D10706D54FF0FF3202FA04F42343ADF84D
:103160002030BDF82030A9F800303CE7202C0FD8E3
:103170000899631E21FA03F3DA0705D54FF0FF32F1
:1031800002FA04F40C430894089BC9F800302AE7BB
:10319000402C2BD0DDE90865611EC4F12102A4F1A9
:1031A000210326FA01F105FA02F225FA03F311438D
:1031B0001943CB0712D50122A4F12003C4F1200149
:1031C00002FA03F322FA01F1A240524243EA010358
:1031D00063EB430332432B43CDE90823DDE90823A6
:1031E000C9E90023FFE66FF00100FCE66FF008007C
:1031F000F9E6082CA0D9102CB3D9202CEED8C3E7BF
:10320000BBF1000FADD0022383E7BBF1000FBBD0B1
:1032100004237EE730B5012A144638BF0124402C30
:1032200085B028BF40240025012ACDE9025518D8D1
:103230001B788DF8083063070AD004AB03EBD40584
:10324000624215F8083C02F00702934005F8083C7A
:10325000009103462246002102A8FFF719FB05B0A2
:1032600030BD082AE4D9102A03D81B88ADF80830ED
:10327000E1E7202A8DBFD3E900231B680293CDE943
:103280000223D8E710B5CB681BB98B600B618B822A
:1032900010BD04691A681C600361C38A013BC382C4
:1032A000CA60F0E703064CBFC0F3C030022070478D
:1032B00008B50246FFF7F6FF022806D15306C2F30F
:1032C0000F2001D100F0030008BDC2F30740FBE767
:1032D0002DE9F04F93B0CDE903230A680446104668
:1032E000FFF7E0FF022814BFC2F306260026002ADB
:1032F0000D46824680F2F78112F0C04940F0F3811A
:10330000097B002900F0EF81022803D02378B34223
:1033100040F0EC81C2F304630693104602F07F0391
:103320000593FFF7C5FF059B29444FEA834848EA08
:103330000A4848EA4668CE7800230022CDE90823EF
:10334000F309834648EA0008029367D0059B00937F
:1033500002466768534608A92046B847002800F08F
:10336000C881276A4FB9414604F10C00FFF7F4FA0F
:10337000074690B96FF0020054E03B6998450DD0C4
:103380003F68002FF9D1414604F10C00FFF7E4FA41
:1033900007460028EED0236A3B60276297F817C0E3
:1033A00006F01F08CCF3840CACEB08001FFA80FE7B
:1033B0000028B8BF0EF12000A8EB0C031FFA83FE13
:1033C000D7E90221B8BF00B2002B0793BEBF0EF1B0
:1033D00020031BB2079352EA010338D0039BDFF8A6
:1033E00024E39A1A049B4FF0000C63EB010196450D
:1033F0007CEB01032BD36B7B97F81AE0734519D153
:10340000029B002B78D0012821DC7868F8B9DFF81E
:10341000F0C2944570EB010316D337E0276A27B951
:103420006FF00C0013B0BDE8F08F3B699845B5D044
:103430003F68F4E7B24890427CEB010301D30020DF
:10344000F0E7029B002BFAD0079B0F2B17DCFA7DCD
:10345000B30002F0030203F07C031343FB7539460B
:103460002046FFF7F9FA6B7BBB76029B3BB9FB7DED
:10347000C3F38402013262F38603FB75D0E76A7BF3
:10348000BB7E9A42DBD1029B002B35D0B309022BC5
:1034900032D0039BBB60049BFB60142200210DA86B
:1034A000FDF7E4FD039B0A93049B0B932B1D0C93E8
:1034B0002B7BADF83EB0013BDBB2ADF83C30069B58
:1034C0008DF84230059B8DF8433094F82C308DF800
:1034D00040A083F001038DF844308DF84180A3684B
:1034E0000AA920469847FB7DC3F38403013303F008
:1034F0001F039B02FB82A2E7FB7DC6F34012B2EBE7
:10350000D31F40F0F980C3F38403434540F0FC80AF
:10351000029A2B7BB609002A52D016F0010661D11F
:10352000032B40F2F480039BBB60049BFB60FB8A8F
:1035300066F30903FB822B7BAE1D033BDBB23246F5
:10354000394604F10C00FFF799FA00280CDA3946E5
:103550002046FFF781FAFB7DC3F38403013303F0B8
:103560001F039B02FB8205E7DDE90884AB883B83F0
:103570004FF6FF73C9F12000A9F1200228FA09F1E2
:1035800004FA00F0014324FA02F211431846C9B2CA
:10359000FFF7B6F909F10809B9F1400F0346E9D17F
:1035A000B8822A7B033AD2B23146FFF7BBF9FB7DE2
:1035B000B882DA43C2F3C01262F3C713FB753EE769
:1035C00086B92E1D013BDBB23246394604F10C00B0
:1035D000FFF754FA0028BADB2A7BB88A013AD2B244
:1035E0003146E2E7F98AC1F30901013B0429DAB265
:1035F0005BD8281D002307F11B069A4208D910F852
:1036000001CB06F801C0013101330529DBB2F4D149
:1036100003990A9104990B91934207F11B010C91B4
:1036200038BF043379680D9134BF55FA83F3002312
:103630000E93FB8AADF83EB0C3F309031A44069B10
:103640008DF84230059B8DF8433094F82C30ADF85E
:103650003C2083F001038DF8443000238DF840A016
:103660008DF841807B602A7BB88A013A291DFFF7DB
:1036700059F93B8BB882834203D1A3680AA920463B
:10368000984720460AA9FFF7FDFDFB7DBA8AC3F3E0
:103690008403013303F01F039B02FB823B8B9A429E
:1036A0000CBF00206FF01000BCE67B68002BAFD091
:1036B000052001E01C3033461E68002EFAD1091A9D
:1036C000081D2E1D184401EB090CBCF11B0F5FFAFD
:1036D00089F39DD89A429BD916F8013B00F8013B2B
:1036E00009F10109EFE76FF009009BE66FF00A00AE
:1036F00098E66FF00B0095E66FF00D0092E600BFC4
:1037000040420F0080841E006FF00E008AE66FF0CA
:103710000F0087E6EFF3098305494A6B22F00102A7
:103720004A63683383F30988002383F31188704761
:1037300000EF00E0302080F3118862B60C4B0D4A98
:10374000D96821F4E0610904090C0A43DA60D3F86E
:10375000FC20094942F08072C3F8FC200A6842F05C
:1037600001020A602022DA7783F82200704700BF46
:1037700000ED00E00003FA05001000E010B5302372
:1037800083F311880E4B5B6813F4006314D0F1EEE1
:10379000103AEFF30984683C4FF08073E361094B02
:1037A000DB6B236684F3098800F0BAFA10B1064B8C
:1037B000A36110BD054BFBE783F31188F9E700BF58
:1037C00000ED00E000EF00E03F03000842030008C6
:1037D000434B4FF4007270B51A605A6912F4C06F0F
:1037E000FBD1404B9A6802F00C02042A20D01A68E0
:1037F00042F480721A601A685205FCD501229A6060
:103800009A6802F00C02042AFAD13749374A0A6052
:103810000A6812F00F02FBD1C3F8982063221A60E5
:103820001A689603FCD42E4A4FF48071C2F88010B7
:10383000C468E50306D51A6842F480321A601A6833
:103840009103FCD5C269D20709D5D3F8982042F07C
:103850000102C3F89820D3F898209607FBD5426957
:10386000DA6044F480721A6004F0807111B11A6851
:103870009501FBD5996802691B4E22F0030501F002
:1038800003012943996085693560316869400907FA
:10389000FBD1134905680D6046684E608068C1F829
:1038A00080006E0417D448698505FCD4996802F03D
:1038B000030021F00301014399609200996851408F
:1038C00011F00C0FFAD1E2055EBF1A6822F4807283
:1038D0001A60002070BD48698005FCD5E6E700BF8E
:1038E000007000400010024000200240000604006A
:1038F00008B500F083F9BDE8084000F05BB90000AE
:1039000010B5394C3948A36A4FF0FF32A262A36A5E
:103910000023A362A16AE16A61F07F01E162E16ACA
:1039200001F07F01E162E16A216B2263216B236375
:10393000216BA16BA263A16BA363A16BE16BE2633B
:10394000E16BE363E16B216C2264226C2364226CE3
:10395000226E42F001022266D4F8802022F0010299
:10396000C4F88020D4F88020A26D42F08052A26575
:10397000A26F22F08052A267A26F1D4A4FF400414D
:103980009160D360136253629362D3621363536393
:103990009363D363136453649364D364136553656F
:1039A000116841F480711160D4F8902012F4407FC6
:1039B0001EBF4FF48032C4F89020C4F890300D4AF6
:1039C0000023A360C4F88820C4F89C30FFF700FFF0
:1039D00010B1094800F0DAF9D4F8903023F003234D
:1039E000C4F8903010BD00BF00100240C448000869
:1039F0000070004055010051BC480008014B53F8CD
:103A00002000704718230020074A08B5536903F0C7
:103A10000103536123B1054A13680BB150689847FD
:103A2000BDE80840FFF7AABE00040140D4500020C2
:103A3000074A08B5536903F00203536123B1054AED
:103A400093680BB1D0689847BDE80840FFF796BE71
:103A500000040140D4500020074A08B5536903F020
:103A60000403536123B1054A13690BB150699847A8
:103A7000BDE80840FFF782BE00040140D45000209A
:103A8000074A08B5536903F00803536123B1054A97
:103A900093690BB1D0699847BDE80840FFF76EBE47
:103AA00000040140D4500020074A08B5536903F0D0
:103AB0001003536123B1054A136A0BB1506A98474A
:103AC000BDE80840FFF75ABE00040140D450002072
:103AD000164B10B55C6904F478725A61A30604D5DC
:103AE000134A936A0BB1D06A9847600604D5104A0E
:103AF000136B0BB1506B9847210604D50C4A936B9E
:103B00000BB1D06B9847E20504D5094A136C0BB191
:103B1000506C9847A30504D5054A936C0BB1D06C43
:103B20009847BDE81040FFF729BE00BF00040140E0
:103B3000D4500020194B10B55C6904F47C425A61E2
:103B4000620504D5164A136D0BB1506D98472305D5
:103B500004D5134A936D0BB1D06D9847E00404D59A
:103B60000F4A136E0BB1506E9847A10404D50C4A4E
:103B7000936E0BB1D06E9847620404D5084A136F58
:103B80000BB1506F9847230404D5054A936F0BB1CE
:103B9000D06F9847BDE81040FFF7F0BD000401402A
:103BA000D450002008B500F0F3FCBDE80840FFF752
:103BB000E5BD0000062108B5084600F033F80621EF
:103BC000072000F02FF80621082000F02BF806212E
:103BD000092000F027F806210A2000F023F806212A
:103BE000172000F01FF80621282000F01BF8BDE880
:103BF000084007211C2000F015B800004FF0E0231A
:103C0000002258684FF0FF31930003F1604303F541
:103C1000614301329042C3F88010C3F88011F3D29F
:103C20007047000000F1604303F561430901C9B228
:103C300083F80013012200F01F039A4043099B0000
:103C400003F1604303F56143C3F880211A607047B4
:103C500000230375826803691B6899689142FBD24F
:103C60005A68036042601060586070470023037513
:103C7000826803691B6899689142FBD85A6803609F
:103C8000426010605860704708B50846302383F3DF
:103C900011880B7D032B05D0042B0DD02BB983F39A
:103CA000118808BD8B6900221A604FF0FF338361D1
:103CB000FFF7CEFF0023F2E7D1E9003213605A602C
:103CC000F3E70000FFF7C4BF054BD9680875186813
:103CD00002681A60536001220275D860FCF71ABBB3
:103CE000484E002030B50C4BDD684B1C87B00446B5
:103CF0000FD02B46094A684600F02AF92046FFF704
:103D0000E3FF009B13B1684600F02CF9A86907B0E7
:103D100030BDFFF7D9FFF9E7484E0020893C000885
:103D2000044B1A68DB6890689B68984294BF002037
:103D300001207047484E0020084B10B51C68D86819
:103D400022681A60536001222275DC60FFF78EFF43
:103D500001462046BDE81040FCF7DCBA484E002082
:103D600038B5074C074908480123002523706560D2
:103D700000F03CFC0223237085F3118838BD00BF9E
:103D8000B0500020E8480008484E002008B572B640
:103D9000044B186500F0ACFA00F05CFB024B032208
:103DA0001A70FEE7484E0020B050002000F010B915
:103DB0008B60022308618B82084670478368A3F1F9
:103DC000840243F8142C026943F8442C426943F8F6
:103DD000402C094A43F8242CC26843F8182C0222CC
:103DE00003F80C2C002203F80B2C044A43F8102C87
:103DF000A3F12000704700BF2D030008484E0020AB
:103E000008B5FFF7DBFFBDE80840FFF75BBF000028
:103E1000024BDB6898610F20FFF756BF484E002029
:103E2000302383F31188FFF7F3BF000008B5014684
:103E3000302383F311880820FFF754FF002383F316
:103E4000118808BD10B503689C68A2420CD85C6854
:103E50008A600B604C602160596099688A1A9A6088
:103E60004FF0FF33836010BD1B68121BECE70000AE
:103E70000A2938BF0A2170B504460D460A26601982
:103E800000F0AEFB00F09AFB041BA54203D8751CA2
:103E90002E460446F3E70A2E04D9BDE870400120FF
:103EA00000F0E4BB70BD0000F8B5144B0D46D961BD
:103EB00003F1100141600A2A1969826038BF0A22A1
:103EC000016048601861A818144600F07BFB0A27BF
:103ED00000F074FB431BA342064606D37C1C281942
:103EE00000F07EFB27463546F2E70A2F04D9BDE8ED
:103EF000F840012000F0BABBF8BD00BF484E0020DA
:103F0000F8B506460D4600F059FB0F4A134653F824
:103F1000107F9F4206D12A4601463046BDE8F84050
:103F2000FFF7C2BFD169BB68441A2C1928BF2C46C1
:103F3000A34202D92946FFF79BFF22463146034898
:103F4000BDE8F840FFF77EBF484E0020584E0020E5
:103F500010B4C0E9032300235DF8044B4361FFF76D
:103F6000CFBF000010B5194C236998420DD0D0E99D
:103F70000032816813605A609A680A449A6000238C
:103F800003604FF0FF33A36110BD2346026843F87E
:103F9000102F53600022026022699A4203D1BDE8CB
:103FA000104000F017BB936881680B44936000F0E9
:103FB00005FB2269E1699268441AA242E4D91144DE
:103FC000BDE81040091AFFF753BF00BF484E00205C
:103FD0002DE9F047DFF8BC8008F110072C4ED8F827
:103FE000105000F0EBFAD8F81C40AA68031B9A4264
:103FF0003ED81444D5E900324FF00009C8F81C40FF
:1040000013605A60C5F80090D8F81030B34201D15F
:1040100000F0E0FA89F31188D5E903312846984782
:10402000302383F311886B69002BD8D000F0C6FAD7
:104030006A69A0EB04094A4582460DD2022000F0CD
:1040400015FB0022D8F81030B34208D1514628465B
:10405000BDE8F047FFF728BF121A2244F2E712EB3F
:10406000090938BF4A4629463846FFF7EBFEB5E74F
:10407000D8F81030B34208D01444211AC8F81C00F4
:10408000A960BDE8F047FFF7F3BEBDE8F08700BFC9
:10409000584E0020484E002038B500F08FFA054AEF
:1040A000D2E90845031B181945F10001C2E90801CE
:1040B00038BD00BF484E002000207047FEE70000DA
:1040C000704700004FF0FF3070470000BFF34F8F84
:1040D000024A1369DB03FCD4704700BF0020024092
:1040E00008B5094B1B7873B9FFF7F0FF074B5A6906
:1040F000002ABFBF064A9A6002F188329A601A68A5
:1041000022F480621A6008BDC850002000200240DE
:104110002301674508B50B4B1B7893B9FFF7D6FF12
:10412000094B5A6942F000425A611A6842F48052BF
:104130001A601A6822F480521A601A6842F4806287
:104140001A6008BDC8500020002002407F289ABF96
:1041500000F58030C0020020704700004FF400607E
:1041600070470000802070477F2808B50BD8FFF704
:10417000EDFF00F500630268013204D10430834290
:10418000F9D1012008BD0020FCE700007F2810B510
:1041900004461FD8FFF79AFFFFF7A2FF0E4BF3224A
:1041A0001A6102225A615A6942EAC0025A615A6986
:1041B00042F480325A61FFF789FF4FF40061FFF744
:1041C000C5FF00F043F9FFF7A5FF2046BDE810400A
:1041D000FFF7CABF002010BD002002402DE9F843C0
:1041E00040EA020313F00703144606D0304B40F2B6
:1041F00082321A600020BDE8F88385182D4A954266
:104200000CD92B4A40F287311160F3E7031D1B687C
:104210004A68934208D1083C08300831072C14D969
:1042200002680B689A42F1D0FFF75AFFFFF74EFF82
:10423000214E08314FF001084FF00009012CA1F187
:10424000080706D8FFF766FF01E0002CECD101203B
:10425000D1E7C6F81480054651F8083C45F8043B00
:1042600051F8043C4360FFF731FF336943F0010329
:104270003361C6F81490026851F8083C9A420CD099
:104280000B4B40F2AF321A600C4B18600C4B1C60A9
:104290000C4B1F60FFF73EFFACE72D6851F8043C64
:1042A0009D4201F10801EBD1083C0830C6E700BF90
:1042B000C45000200000040800200240B850002034
:1042C000C0500020BC500020084908B50B7828B128
:1042D0001BB9FFF705FF01230B7008BD002BFCD0B5
:1042E000BDE808400870FFF715BF00BFC8500020A8
:1042F00008B50649064800F0ABF8BDE808404FF4A1
:1043000080414FF0805000F0A3B800BF007F010053
:1043100000010020084600F033BA000038B5EFF382
:1043200011859DB9EFF30584C4F30804302334B13B
:1043300083F31188FFF7B0FE85F3118838BD83F34E
:104340001188FFF7A9FE84F3118838BDBDE8384015
:10435000FFF7A2BE38B5FFF7E1FF114C114AC008C4
:1043600040EA4170A0FB025EC908A0FB040C1CEBF4
:10437000050CA1FB04404FF000035B41A1FB0212BE
:104380001CEB040C43EB000011EB0E0142F10002A8
:10439000411842F10000090941EA007038BD00BF30
:1043A000CFF753E3A59BC4200244D2B2904200D180
:1043B0007047431C800000F1804000F514500068F5
:1043C00041F8040BD8B2F1E7124B10B5D3F8904086
:1043D000240409D4D3F89040C3F89040D3F8904017
:1043E00044F40044C3F890400B4C2368024443F467
:1043F00080732360D2B2904200D110BD431C800074
:1044000000F1804000F5145051F8044B0460D8B21C
:10441000F1E700BF001002400070004007B5012224
:1044200001A90020FFF7C0FF019803B05DF804FB6D
:1044300013B50446FFF7F2FFA04205D0012201A9FF
:1044400000200194FFF7C0FF02B010BD70470000CC
:104450007047000070470000074B45F255521A6044
:1044600003225A6040F2FF729A604CF6CC421A6006
:10447000024B01221A70704700300040D0500020DB
:10448000034B1B781BB1034B4AF6AA221A607047F4
:10449000D050002000300040054B1A6832B902F1BC
:1044A000804202F50432D2F894201A60704700BFAF
:1044B000CC500020024B4FF40002C3F89420704708
:1044C0000010024008B5FFF7E7FF024B1868C0F381
:1044D000407008BDCC50002070470000FEE700008F
:1044E0000A4B0B480B4A90420BD30B4BDA1C121AA7
:1044F000C11E22F003028B4238BF00220021FCF7CC
:10450000B5BD53F8041B40F8041BECE76C4A0008E7
:104510005451002054510020545100200023054ADA
:1045200019460133102BC2E9001102F10802F8D13B
:10453000704700BFD450002008B5124B9A6D42F06E
:1045400001029A659A6F42F001029A670E4A9B6FC8
:10455000936843F0010393600620FFF74FFA0B4B7B
:10456000B0FBF3F04FF080434FF0FF320138986218
:10457000DA6200229A615A63DA605A6001225A6153
:104580001A6008BD00100240002004E040420F0005
:104590004FF0804208B51169D3680B40D9B2C943C6
:1045A0009B07116107D5302383F31188FFF7FEFBCA
:1045B000002383F3118808BDFFF7BEBF4FF080438F
:1045C000586A70474FF08043002258631A610222F4
:1045D000DA6070474FF080430022DA6070470000D5
:1045E0004FF0804358637047FEE7000070B51B4BE7
:1045F00001630025044686B0586085620E46FFF7C9
:1046000099F804F11003C4E904334FF0FF33C4E90F
:104610000635C4E90044A560E562FFF7CFFF2B46ED
:104620000246C4E9082304F134010D4A25658023BC
:104630002046FFF7BDFB0123E0600A4A03750092A4
:1046400072680192B268CDE90223074B6846CDE952
:104650000435FFF7D5FB06B070BD00BFB050002099
:10466000F4480008F9480008E9450008024AD36AFE
:104670001843D062704700BF484E00204B6843602B
:104680008B688360CB68C3600B6943614B690362CD
:104690008B6943620B6803607047000008B5204BCC
:1046A000DA6A42F07F02DA62DA6A22F07F02DA62C4
:1046B000DA6ADA6C42F07F02DA64DA6E42F07F0284
:1046C000DA66184ADB6E11464FF09040FFF7D6FFCE
:1046D00002F11C0100F58060FFF7D0FF02F1380104
:1046E00000F58060FFF7CAFF02F1540100F5806019
:1046F000FFF7C4FF02F1700100F58060FFF7BEFF15
:1047000002F18C0100F58060FFF7B8FF02F1A8010B
:1047100000F58060FFF7B2FFBDE80840FFF7F0B892
:10472000001002400049000808B500F009F8FFF742
:1047300017FBBDE80840FFF7AFBE00007047000060
:1047400008B5FFF7D5F8FFF7E9FEFFF7F7FFBDE87B
:104750000840FFF731BF00000B460146184600F045
:1047600001B8000010B5054C13462CB10A460146AD
:104770000220AFF3008010BD2046FCE700000000DF
:10478000024B01461868FFF7C5BD00BF402300205B
:1047900010B501390244904201D1002005E00378B0
:1047A00011F8014FA34201D0181B10BD0130F2E7F0
:1047B0002DE9F041A3B1C91A17780144044603F169
:1047C000FF3C8C42204601D9002009E00578BD421B
:1047D00004F10104F5D10CEB0405D618A54201D172
:1047E000BDE8F08115F8018D16F801EDF045F5D022
:1047F000E7E70000034611F8012B03F8012B002A1C
:10480000F9D17047696E2E73696572726161657264
:104810006F73706163652E547275654E6176507268
:104820006F2D47340000000040A2E4F16468910657
:104830000041A3E5F265699207000000426164202F
:1048400043414E496661636520696E6465782E0058
:104850000000000000000000551E0008E5180008D8
:104860006D2500085519000861190008AD1B0008E6
:10487000051B00081D19000821190008F918000877
:10488000E1180008691B000805190008F526000852
:10489000A5260008111900083D1B000801040E059B
:1048A000054B02020E05054B04010E05054B0501E3
:1048B0000B04044B0801060303460000636C6B7392
:1048C000776300000003000000000000000100000A
:1048D0000000010103000000132831010407040057
:1048E0000100000063300000E4480008A04E0020F2
:1048F000B05000206D61696E0069646C6500000055
:104900001001942A000000009AAAAAAA0000142408
:10491000FBFF000000000000009009000004000000
:1049200000000000AAA6AAAA00000000DFFF000005
:104930000000000000000000000000000000000077
:10494000AAAAAAAA00000000FFFF000000000000C1
:10495000000000000000000000000000AAAAAAAAAF
:1049600000000000FFFF0000000000000000000049
:104970000000000000000000AAAAAAAA000000008F
:10498000FFFF000000000000000000000000000029
:1049900000000000AAAAAAAA00000000FFFF000071
:1049A0000000000000000000000000000000000007
:1049B000AAAAAAAA00000000FFFF00000000000051
:1049C0000000000000000000B5140000000000001E
:1049D0000070030000000000FE2A0100D204000065
:1049E000006889096D8BB90200B4C40400688909A4
:1049F00000688909006889090068890900688909CF
:104A00000068890900000000442300200000000025
:104A10000000000000000000000000000000000096
:104A20000000000000000000000000000000000086
:104A30000000000000000000000000000000000076
:104A40000000000000000000000000000000000066
:104A50000000000000000000000000000000000056
:0C4A60000000000000000000000000004A
:00000001FF
